:020000040000FA
:100000000000000000000000000000000000003FB1
:100010003838380000000000000000000000003FF9
:100020000707070000000000000000000000003F7C
:100030003F3F3F0000000000000000000000003FC4
:100040000000003838383800000000000000003F91
:100050003838383838383800000000000000003FD9
:100060000707073838383800000000000000003F5C
:100070003F3F3F3838383800000000000000003FA4
:100080000000000707070700000000000000003F15
:100090003838380707070700000000000000003F5D
:1000A0000707070707070700000000000000003FE0
:1000B0003F3F3F0707070700000000000000003F28
:1000C0000000003F3F3F3F00000000000000003FF5
:1000D0003838383F3F3F3F00000000000000003F3D
:1000E0000707073F3F3F3F00000000000000003FC0
:1000F0003F3F3F3F3F3F3F00000000000000003F08
:100100000000000000000038383800000000003F08
:100110003838380000000038383800000000003F50
:100120000707070000000038383800000000003FD3
:100130003F3F3F0000000038383800000000003F1B
:100140000000003838383838383800000000003FE8
:100150003838383838383838383800000000003F30
:100160000707073838383838383800000000003FB3
:100170003F3F3F3838383838383800000000003FFB
:100180000000000707070738383800000000003F6C
:100190003838380707070738383800000000003FB4
:1001A0000707070707070738383800000000003F37
:1001B0003F3F3F0707070738383800000000003F7F
:1001C0000000003F3F3F3F38383800000000003F4C
:1001D0003838383F3F3F3F38383800000000003F94
:1001E0000707073F3F3F3F38383800000000003F17
:1001F0003F3F3F3F3F3F3F38383800000000003F5F
:100200000000000000000000000000000000003FAF
:100210000004040404040004000000000000003F87
:1002200000000A0A0A000000000000000000003F71
:10023000000A0A1F0A1F0A0A000000000000003F0F
:1002400000040F140E051E04000000000000003F13
:100250000018190204081303000000000000003F0A
:1002600000040A0A0C15120D000000000000003FF7
:100270000004040800000000000000000000003F2F
:100280000002040808080402000000000000003F0B
:100290000008040202020408000000000000003F01
:1002A0000004150E040E1504000000000000003FBD
:1002B000000004041F040400000000000000003FD0
:1002C0000000000000000808100000000000003FCF
:1002D000000000000E000000000000000000003FD1
:1002E0000000000000000C0C000000000000003FB7
:1002F0000000010204081000000000000000003FA0
:10030000000E11111511110E000000000000003F39
:1003100000040C040404040E000000000000003F70
:10032000000E11010608101F000000000000003F31
:10033000001F01020601110E000000000000003F36
:100340000002060A121F0202000000000000003F27
:10035000001F101E0101110E000000000000003FF0
:10036000000708101E11110E000000000000003FE1
:10037000001F010204080808000000000000003F00
:10038000000E11110E11110E000000000000003FC0
:10039000000E11110F01021C000000000000003FC0
:1003A0000000000008000008000000000000003FFE
:1003B0000000000800000808100000000000003FD6
:1003C0000002040810080402000000000000003FC2
:1003D0000000001F001F0000000000000000003FA0
:1003E0000008040201020408000000000000003FB1
:1003F000000E110102040004000000000000003F94
:100400000002041F101E101F000000000000003F2B
:1004100000040A111F111111000000000000003F2C
:10042000001E11111E11111E000000000000003FEF
:10043000000E11101010110E000000000000003F0F
:10044000001E09090909091E000000000000003F04
:10045000001F10101E10101F000000000000003FC1
:10046000001F10101E101010000000000000003FC0
:10047000000E11101013110F000000000000003FCB
:10048000001111111F111111000000000000003FA8
:10049000000E04040404040E000000000000003FED
:1004A000000202020202120C000000000000003FE5
:1004B0000011121418141211000000000000003F77
:1004C000000808080808080F000000000000003FAE
:1004D00000111B1515111111000000000000003F54
:1004E0000011111915131111000000000000003F48
:1004F000000E11111111110E000000000000003F4C
:10050000001E11111E101010000000000000003F1E
:10051000000E11111115120D000000000000003F27
:10052000001E11111E141211000000000000003FF7
:10053000000E11100E01110E000000000000003F1F
:10054000001F040404040404000000000000003F35
:10055000001111111111110E000000000000003FE8
:10056000001111110A0A0404000000000000003FFD
:10057000001111111515150A000000000000003FC0
:100580000011110A040A1111000000000000003FD0
:100590000011110A04040404000000000000003FE0
:1005A000001F01020408101F000000000000003FAF
:1005B00000070C141F141417000000000000003F77
:1005C00000010E1315190E10000000000000003F7E
:1005D0000004000E111F1111000000000000003F78
:1005E000000A00111111110E000000000000003F70
:1005F000000000000000001F000000000000003F9D
:100600000002040E111F100E000000000000003F49
:100610000000000E010F110F000000000000003F5D
:100620000010101E1111111E000000000000003FFC
:100630000000000F1010100F000000000000003F2D
:100640000001010F1111110F000000000000003F18
:100650000000000E111F100E000000000000003FFF
:10066000000204040E040404000000000000003F27
:100670000000000F1111110F010E00000000003FDB
:100680000010101E11111111000000000000003FA9
:100690000004000C0404040E000000000000003FF1
:1006A0000004000C04040404040800000000003FDF
:1006B000000808090A0C0A09000000000000003FB9
:1006C000000C04040404040E000000000000003FBD
:1006D0000000001A15151515000000000000003F6D
:1006E0000000001E11111111000000000000003F69
:1006F0000000000E1111110E000000000000003F6C
:100700000000001E1111111E101000000000003F1B
:100710000000000F1111110F010100000000003F47
:100720000000000B0C080808000000000000003F5B
:100730000000000F100E011E000000000000003F2E
:100740000000040E04040402000000000000003F4A
:10075000000000111111110F000000000000003F07
:1007600000000011110A0A04000000000000003F10
:10077000000000111111150A000000000000003FE8
:10078000000000110A040A11000000000000003FF0
:10079000000000111111110F010E00000000003FB8
:1007A0000000001F0204081F000000000000003FBE
:1007B0000000001A050F140F000000000000003FA9
:1007C0000000010E1315190E100000000000003F7C
:1007D0000004000E010F110F000000000000003F98
:1007E00000000A001111110F000000000000003F7E
:1007F000001F1F1F1F1F1F1F000000000000003FE1
:100800000000000000000007070700000000003F94
:100810003838380000000007070700000000003FDC
:100820000707070000000007070700000000003F5F
:100830003F3F3F0000000007070700000000003FA7
:100840000000003838383807070700000000003F74
:100850003838383838383807070700000000003FBC
:100860000707073838383807070700000000003F3F
:100870003F3F3F3838383807070700000000003F87
:100880000000000707070707070700000000003FF8
:100890003838380707070707070700000000003F40
:1008A0000707070707070707070700000000003FC3
:1008B0003F3F3F0707070707070700000000003F0B
:1008C0000000003F3F3F3F07070700000000003FD8
:1008D0003838383F3F3F3F07070700000000003F20
:1008E0000707073F3F3F3F07070700000000003FA3
:1008F0003F3F3F3F3F3F3F07070700000000003FEB
:10090000000000000000003F3F3F00000000003FEB
:10091000383838000000003F3F3F00000000003F33
:10092000070707000000003F3F3F00000000003FB6
:100930003F3F3F000000003F3F3F00000000003FFE
:10094000000000383838383F3F3F00000000003FCB
:10095000383838383838383F3F3F00000000003F13
:10096000070707383838383F3F3F00000000003F96
:100970003F3F3F383838383F3F3F00000000003FDE
:10098000000000070707073F3F3F00000000003F4F
:10099000383838070707073F3F3F00000000003F97
:1009A000070707070707073F3F3F00000000003F1A
:1009B0003F3F3F070707073F3F3F00000000003F62
:1009C0000000003F3F3F3F3F3F3F00000000003F2F
:1009D0003838383F3F3F3F3F3F3F00000000003F77
:1009E0000707073F3F3F3F3F3F3F00000000003FFA
:1009F0003F3F3F3F3F3F3F3F3F3F00000000003F42
:100A00000000000000000000000000000000003FA7
:100A10000004040404040004000000000000003F7F
:100A200000000A0A0A000000000000000000003F69
:100A3000000A0A1F0A1F0A0A000000000000003F07
:100A4000000000110E0A0E11000000000000003F1F
:100A50000018190204081303000000000000003F02
:100A600000040A0A0C15120D000000000000003FEF
:100A70000004040800000000000000000000003F27
:100A80000002040808080402000000000000003F03
:100A90000008040202020408000000000000003FF9
:100AA0000004150E040E1504000000000000003FB5
:100AB000000004041F040400000000000000003FC8
:100AC0000000000000000808100000000000003FC7
:100AD000000000000E000000000000000000003FC9
:100AE0000000000000000C0C000000000000003FAF
:100AF0000000010204081000000000000000003F98
:100B0000000E11111511110E000000000000003F31
:100B100000040C040404040E000000000000003F68
:100B2000000E11010608101F000000000000003F29
:100B3000001F01020601110E000000000000003F2E
:100B40000002060A121F0202000000000000003F1F
:100B5000001F101E0101110E000000000000003FE8
:100B6000000708101E11110E000000000000003FD9
:100B7000001F010204080808000000000000003FF8
:100B8000000E11110E11110E000000000000003FB8
:100B9000000E11110F01021C000000000000003FB8
:100BA0000000000008000008000000000000003FF6
:100BB0000000000800000808100000000000003FCE
:100BC0000002040810080402000000000000003FBA
:100BD0000000001F001F0000000000000000003F98
:100BE0000008040201020408000000000000003FA9
:100BF000000E110102040004000000000000003F8C
:100C00000002041F101E101F000000000000003F23
:100C100000040A111F111111000000000000003F24
:100C2000001E11111E11111E000000000000003FE7
:100C3000000E11101010110E000000000000003F07
:100C4000001E09090909091E000000000000003FFC
:100C5000001F10101E10101F000000000000003FB9
:100C6000001F10101E101010000000000000003FB8
:100C7000000E11101013110F000000000000003FC3
:100C8000001111111F111111000000000000003FA0
:100C9000000E04040404040E000000000000003FE5
:100CA000000202020202120C000000000000003FDD
:100CB0000011121418141211000000000000003F6F
:100CC000000808080808080F000000000000003FA6
:100CD00000111B1515111111000000000000003F4C
:100CE0000011111915131111000000000000003F40
:100CF000000E11111111110E000000000000003F44
:100D0000001E11111E101010000000000000003F16
:100D1000000E11111115120D000000000000003F1F
:100D2000001E11111E141211000000000000003FEF
:100D3000000E11100E01110E000000000000003F17
:100D4000001F040404040404000000000000003F2D
:100D5000001111111111110E000000000000003FE0
:100D6000001111110A0A0404000000000000003FF5
:100D7000001111111515150A000000000000003FB8
:100D80000011110A040A1111000000000000003FC8
:100D90000011110A04040404000000000000003FD8
:100DA000001F01020408101F000000000000003FA7
:100DB000000A000E111F1111000000000000003F8A
:100DC000000A000E1111110E000000000000003F8B
:100DD0000004000E111F1111000000000000003F70
:100DE000000A00111111110E000000000000003F68
:100DF000000000000000001F000000000000003F95
:100E00000002040E111F100E000000000000003F41
:100E10000000000E010F110F000000000000003F55
:100E20000010101E1111111E000000000000003FF4
:100E30000000000F1010100F000000000000003F25
:100E40000001010F1111110F000000000000003F10
:100E50000000000E111F100E000000000000003FF7
:100E6000000204040E040404000000000000003F1F
:100E70000000000F1111110F010E00000000003FD3
:100E80000010101E11111111000000000000003FA1
:100E90000004000C0404040E000000000000003FE9
:100EA0000004000C04040404040800000000003FD7
:100EB000000808090A0C0A09000000000000003FB1
:100EC000000C04040404040E000000000000003FB5
:100ED0000000001A15151515000000000000003F65
:100EE0000000001E11111111000000000000003F61
:100EF0000000000E1111110E000000000000003F64
:100F00000000001E1111111E101000000000003F13
:100F10000000000F1111110F010100000000003F3F
:100F20000000000B0C080808000000000000003F53
:100F30000000000F100E011E000000000000003F26
:100F40000000040E04040402000000000000003F42
:100F5000000000111111110F000000000000003FFF
:100F600000000011110A0A04000000000000003F08
:100F7000000000111111150A000000000000003FE0
:100F8000000000110A040A11000000000000003FE8
:100F9000000000111111110F010E00000000003FB0
:100FA0000000001F0204081F000000000000003FB6
:100FB000000A000E010F110F000000000000003FAA
:100FC00000000A000E11110E000000000000003F9A
:100FD0000004000E010F110F000000000000003F90
:100FE00000000A001111110F000000000000003F76
:100FF000001F1F1F1F1F1F1F000000000000003FD9
:00000001FF
